:1000000020308400493009208A11342D04068001F3
:0C001000840A0406031D06286400003466
:10073A00F90000307A1879070310F90D0310FA0C42
:10074A00FA08031908009F2B8301BF0083160317B9
:10075A008C18AB2B831203133F0803178D008316E3
:10076A008C130C1483120C08031308008301C000B5
:10077A00831603178C18BD2B831203134008031723
:10078A008D0003133F0803178C0083168C13031084
:10079A008B1B03148B130C1555308D00AA308D005A
:1007AA008C140C1103188B17830108000430830181
:1007BA00C100FA300000FF3E031DDF2B6400C10BAD
:1007CA00DE2BFF30BF07031CC00340083F04031998
:1007DA000800DB2B8301C1000430C200FA3000009C
:1007EA00FF3E031DF42B6400C20BF32BC10BF12B4C
:1007FA0008008301BF000430C000FA30EF23640010
:10080A00C00B022CBF0B002C08008301C80048084B
:10081A0093008316141C0E2C8312130808008301FC
:10082A00B501B50AB601222C061035080A240F3084
:10083A000A240614B50A0319B60A3608803AF900DA
:10084A008030790207300319350203180800192C81
:10085A008301BF0006100A300A243F080A2406143E
:10086A0008008301061009300A24FF300A240614FE
:10087A0005302D248A1106100B300A2405300A246B
:10088A00061406100C300A2401300A240614061035
:10089A000F300A2401300A24061486160230FE2379
:1008AA0006100F300A2400300A24061486120800A3
:1008BA008301051908008612061009300A2401303E
:1008CA000A240614061001300A240B300A240614DE
:1008DA00061002300A2405300A24061406100330D2
:1008EA000A2405300A240614061004300A241D308E
:1008FA000A240614061005300A2405300A240614B0
:10090A00061006300A2400300A240614080083015F
:10091A00051908008612061009300A2421300A2413
:10092A000614061001300A240E300A240614061092
:10093A0002300A2400300A240614061003300A245E
:10094A0047300A240614061004300A2477300A2491
:10095A000614061005300A2406300A240614061066
:10096A0006300A240D300A24061408008301C70041
:10097A00061009300A24FF300A2406140A30FA0045
:10098A0047088A1190278A11C1000A304702031CBE
:10099A00D62C0A30FA0041088A119D238A1147028F
:1009AA00D72C4708C2000A30FA003F088A1190275C
:1009BA008A11C3000A303F02031CEB2C0A30FA00EA
:1009CA0043088A119D238A113F02EC2C3F08C40078
:1009DA000A30FA0040088A1190278A11C5000A30A5
:1009EA004002031C002D0A30FA0045088A119D2393
:1009FA008A114002012D4008C600061001300A245F
:100A0A0041080A240614061002300A244208803ECD
:100A1A000A240614061003300A2443080A2406147A
:100A2A00061004300A244408803E0A2406140610DC
:100A3A0005300A2445080A240614061006300A243A
:100A4A0046080A240614080083160313861406119E
:100A5A000612403094002130831294000800831655
:100A6A0003139B018312850186011F3083168500BB
:100A7A008612061029253624BB01BC01BD01BE0120
:100A8A00B101B301B001AE01B701B801A201A001E1
:100A9A00B201B401A601AC01AD0100308A11A9234B
:100AAA008A11B900BA01390A3A04031D652DB90140
:100ABA00B90ABA01BF01BF0A00308A11BB238A11E1
:100ACA002230BF003830C0000C30BB248A11851890
:100ADA006C2D851C6E2DB70A0319B80A3808803A9E
:100AEA00F90080307902793003193702031C802D0E
:100AFA005D248A11B101AF080319E82DAF01AB08D3
:100B0A000319892DAB01E32D0519912D2D08BF007D
:100B1A00C0012C08BB248A112C08A2002D08A300AE
:100B2A003208A5003408A4002608A100A208031D63
:100B3A00A12D00302D248A1109302202031CA82D70
:100B4A0005302D248A1116302202031CAE2D0030E6
:100B5A002D240A30FB000030FC01A30803190130E0
:100B6A00F900FA018A117B278A117A087904031994
:100B7A00D92D390A3A04031DC52DB901B90ABA019A
:100B8A002208BF0039088A11BB232308BF00390A8B
:100B9A008A11BB230230B9070318BA0A3908BF0001
:100BAA0000308A11BB238A112A0C031CDE2D8616FB
:100BBA00DF2D861283120313B101B10AB701B801FE
:100BCA00B001B301AE01A00A0519B101B1080319B8
:100BDA00F92D3C3020020318F92D2308BF00200804
:100BEA00C0002208BB248A116430EF23A701B50193
:100BFA00B50AB6013608803AF900803079026530C4
:100C0A00031935020318112E8518A70A0130EF239C
:100C1A00B50A0319B60AFF2DA801B501B50AB6012E
:100C2A003608803AF90080307902653003193502B6
:100C3A000318272E8518A80A0130EF23B50A0319CD
:100C4A00B60A152EA901B501B50AB6013608803AC9
:100C5A00F9008030790265300319350203183D2EF8
:100C6A008518A90A0130EF23B50A0319B60A2B2EF3
:100C7A00051D462E2808BF002908C0002708BB24E6
:100C8A008A111F302702A7010318A70A1F3028025A
:100C9A00A8010318A80A1F302902A9010318A90AE2
:100CAA00A90803195E2EAC01AD01B201B401A60177
:100CBA00A0012C30BF000130C000DB233F2FA70862
:100CCA0003196C2D5030862EA70803196C2D283075
:100CDA00862EA70803196C2D1430862EA70803192F
:100CEA006C2D0A30862EA70803196C2D0830862E23
:100CFA00A70803196C2D0430862EA70803196C2D3A
:100D0A000230B2078C2EA70803196C2DB20AB30A57
:100D1A006C2DA70803196C2D0A30A12EA7080319F8
:100D2A006C2D0830A12EA70803196C2D0430A12EB2
:100D3A00A70803196C2D0230B407C62EA708031999
:100D4A006C2DB40AC62EA70803196C2D1430C02EB8
:100D5A00A70803196C2D0A30C02EA70803196C2D99
:100D6A000830C02EA70803196C2D0430C02EA7081E
:100D7A0003196C2D0230A607C62EA70803196C2D7D
:100D8A00A60AAE0A6C2DA70803196C2D1430E02EA2
:100D9A00A70803196C2D0A30E02EA70803196C2D39
:100DAA000830E02EA70803196C2D0430E02EA7089E
:100DBA0003196C2D0230AC070A2FA70803196C2DF2
:100DCA00AC0A0A2FA70803196C2D2830042FA7088C
:100DDA0003196C2D1430042FA70803196C2D0A303F
:100DEA00042FA70803196C2D0830042FA70803192C
:100DFA006C2D0430042FA70803196C2D0230AD079F
:100E0A000A2FA70803196C2DAD0AB00A6C2D051913
:100E1A006C2D0230FB00FC012808F900FA013308A6
:100E2A00292F05196C2D0230FB00FC012808F90056
:100E3A00FA012E08292F05196C2D0230FB00FC013E
:100E4A002808F900FA013008F9070318FA0A8A1182
:100E5A007B278A117A087904031D6C2D8C248A1148
:100E6A00B101AB01AB0A6C2D2808AA006C2DAF01A9
:100E7A00AF0A6C2D2008F900C43E03186C2D2B3ED6
:100E8A00031C6C2D1130F90207308A0050307907A3
:100E9A0003188A0A8200642E692E6E2E732E782E0B
:100EAA007D2E822E882E8E2E932E982E9D2EA32E48
:100EBA00A82EAD2EB22EB72EBC2EC22E6C2D6C2DA6
:100ECA006C2DC82ECD2ED22ED72EDC2EE22EE72E5A
:100EDA00EC2EF12EF62EFB2E002F062F6C2D6C2DEC
:100EEA000C2F162F6C2D202F392F3C2FFF01FA1FA4
:100EFA00852FF909F90A0319FA03FA097F17FF1767
:100F0A007C088039FF06FC1FC72FFB09FB0A03195F
:100F1A00FC03FC09C72FF900FD010310FD307A0715
:100F2A00031CB72FFC01F0307A05031D9F2F0430F4
:100F3A00FC00FA0EFB010310FC0AFA0D031CA12F98
:100F4A00FA0C7A0879020318F900FB0DFC0BA52F9D
:100F5A00FD1FB12FFB09FB0A7B08FD1F0800F909D9
:100F6A00F90A0800FA0C0318C02FFA0C031CF9013D
:100F7A000310F90C031C03107908FB00F901F90DA1
:100F8A00AD2FFF01FD01FE017B087C04031DD02F5C
:100F9A00F901FA0100341F30FF040310FF0AFB0DA8
:100FAA00FC0D031CD32FFC0CFB0C7C087A02031DDE
:100FBA00E02F7B087902031CE82F7B08F9027C08E2
:100FCA00031C7C0AFA02FD0DFE0DFF0BFF1AD82F37
:100FDA00FF1FF42FFD09FD0A0319FE03FE097D0810
:100FEA00FB007E08FC007F1F0034F909F90A031987
:060FFA00FA03FA090034BD
:04400E002A3FFC3F0A
:00000001FF
